S024000062696E2F6F70656E62746C5F6F6C696D65785F73746D3332703130332E737265639B
S315080000005411002011450008FD440008FD4400086D
S31508000010FD440008FD440008FD440008FD440008AE
S31508000020FD440008FD440008FD440008FD4400089E
S31508000030FD440008FD440008FD440008FD4400088E
S31508000040FD440008FD440008FD440008FD4400087E
S31508000050FD440008FD440008FD440008FD4400086E
S31508000060FD440008FD440008FD440008FD4400085E
S31508000070FD440008FD440008FD440008FD4400084E
S31508000080FD440008FD440008FD440008FD4400083E
S31508000090FD440008FD440008FD440008FD4400082E
S315080000A0FD440008FD440008FD440008FD4400081E
S315080000B0FD440008FD440008FD440008FD4400080E
S315080000C0FD440008FD440008FD440008FD440008FE
S315080000D0FD440008FD440008FD440008FD440008EE
S315080000E0FD440008FD440008FD440008FD440008DE
S315080000F0FD440008FD440008FD440008FD440008CE
S31508000100FD440008FD440008FD440008FD440008BD
S31508000110FD440008FD440008FD440008FD440008AD
S31508000120FD440008FD440008FD440008FD4400089D
S31508000130FD440008FD440008FD440008FD4400088D
S31508000140FD440008FD440008FD440008FD4400087D
S3150800015010B572B618481949016019498D46124BEF
S31508000160124A9A4211D202F10403114CE41A24F0FD
S31508000170030404F104044FF0000310460D495A58CD
S315080001801A5003F10403A342F9D10E480E494FF061
S3150800019000028842B8BF40F8042BFFF6FAAF03F016
S315080001A03DF800F0A3F810BD08000020000000206C
S315080001B00B000020C84E000808ED00E0000000080B
S315080001C05411002008000020540F002000B589B003
S315080001D04FF000030093019302930393049305934E
S315080001E0069307930A48694602F09AFE40B9009BAF
S315080001F04BB19DF8080080F01000C0F3001004E031
S315080002004FF0000001E04FF0000009B000BD00BF4C
S3150800021074450008004870477445000808B5084842
S315080002204FF0000380F8243206494FF00A0202F024
S3150800023081FA20B94FF00102014B83F8242208BD48
S31508000240080000209445000838B50A4B93F8243274
S31508000250012B02D1074802F079FD074D4FF0400403
S315080002602846214600F09AFE0028F9D0034802F0F5
S315080002707DFE38BD08000020004400407445000893
S3150800028008B5044B93F82432012B02D1014802F039
S315080002905DFD08BD0800002070B50646114B93F8B1
S315080002A02432012B0BD10F4902F014FF002806DA7D
S315080002B00C484FF0000380F8243202F047FD3178ED
S315080002C079B1094C4FF08005204600F061FE2046C2
S315080002D0294600F063FE0028F9D016F8011F002908
S315080002E0F2D170BD080000200044004000B583B07C
S315080002F04FF0000300930193474B1A6842F001023E
S315080003001A605968454A0A405A601A6822F0847287
S3150800031022F480321A601A6822F480221A605A6817
S3150800032022F4FE025A604FF41F029A601A6842F4D9
S3150800033080321A601A4640F2DC53116801F4003123
S315080003400191009901F101010091019911B90099F2
S315080003509942F2D1304B1B6813F4003F04D1304860
S315080003604FF0760103F018FD2E4B1A6842F0100282
S315080003701A601A6822F003021A601A6842F002022A
S315080003801A60A3F580535A685A605A6842F40052B4
S315080003905A605A6842F480625A605A6822F47C129B
S315080003A05A605A6842F4E8125A601A6842F0807233
S315080003B01A601A6812F0007FFBD0174B5A6822F0B1
S315080003C003025A605A6842F002025A605A6802F0FA
S315080003D00C02082AFAD1104BDA6942F40032DA61C3
S315080003E09A6942F005029A61A3F584331A6822F4E1
S315080003F070621A601A6842F430621A601A6822F447
S3150800040070421A601A6842F480421A6002F0BCFE12
S3150800041002F0C8FEFCE700BF001002400000FFF82B
S31508000420A44500080020024038B50146084800F0F7
S3150800043093FD074D4FF001042846214600F0A2FD22
S315080004400028F9D0024800F089FDC0B238BD00BFC7
S315080004500038004070B503F0D9FD00F5FA764FF084
S31508000460FF052846FFF7E0FF0446FF2803D003F000
S31508000470CDFD8642F5D8FF2C14BF0020012070BDA3
S3150800048010B504464FF0FF00FFF7CEFF207010BDF1
S31508000490F8B504460D4603F0B9FD00F164074FF0C0
S315080004A0FF063046FFF7C0FFFF2806D103F0AEFD72
S315080004B08742F6D84FF00000F8BDFE2816D126462A
S315080004C02046FFF7DDFF04F1010004F10204FFF7FF
S315080004D0D7FF023DF3D14FF0FF00FFF7A5FF4FF01E
S315080004E0FF00FFF7A1FF4FF00100F8BD4FF0000035
S315080004F0F8BD00BF38B505460C46FFF7ABFF38B365
S315080005002046FFF791FFFD2C25D005F1020405F2E0
S31508000510022514F8020CFFF787FF14F8010CFFF701
S3150800052083FF04F10204AC42F3D14FF0FF00FFF75A
S315080005307BFF4FF0FF00FFF777FF4FF0FF00FFF755
S3150800054073FF00F01F00052814BF0020012038BDE6
S315080005504FF0000038BD4FF0010038BD08B505481A
S315080005604FF4805100F0A6FC4FF0FF00FFF75CFF48
S3150800057008BD00BF000C014008B50A484FF4805179
S3150800058000F09AFC4FF0FF00FFF74EFFFFF762FFFF
S3150800059020B9FFF7E3FF4FF0000008BD4FF0010058
S315080005A008BD00BF000C014038B504460D4610F0E2
S315080005B0800F09D04FF037004FF00001FFF7F4FF26
S315080005C0012843D804F07F04FFF7C8FFFFF7D4FFDC
S315080005D078B344F04000FFF727FF4FEA1560FFF7AE
S315080005E023FFC5F30740FFF71FFFC5F30720FFF7F3
S315080005F01BFFE8B2FFF718FF1CB3082C1CD04FF0FE
S315080006000100FFF711FF0C2C03D14FF0FF00FFF795
S315080006100BFF4FF00A044FF0FF052846FFF704FFCB
S3150800062010F0800F12D004F1FF3313F0FF04F4D159
S3150800063038BD4FF0FF0038BD4FF08700FFF7F4FED6
S31508000640E7E74FF09500FFF7EFFEE2E738BD00BF9A
S315080006502DE9F04389B0002840F07881C04B1B781B
S3150800066003F00203DBB213B1BD4B187880E14FF0FB
S3150800067008004FF0010100F021FC4FF480404FF0D4
S31508000680010100F029FC4FF48057ADF800704FF0D7
S3150800069010098DF803904FF003068DF80260B14CEF
S315080006A02046694600F0ACFB2046394600F002FCBD
S315080006B04FF42043ADF800308DF802604FF0180370
S315080006C08DF803302046694600F09AFB4FF48043C4
S315080006D0ADF800304FF048038DF8033020466946E0
S315080006E000F08EFB4FF00005ADF808504FF482730A
S315080006F0ADF80A30ADF80C50ADF80E50ADF8105004
S315080007004FF40073ADF812304FF03803ADF81430DB
S31508000710ADF816504FF00703ADF81830DFF84C82E5
S31508000720404602A900F0E6FB4046294600F01AFCBE
S3150800073040464FF0010100F0FFFB2046394600F025
S31508000740B9FB4FF40045ADF804508DF806608DF8F6
S315080007500790204601A900F053FB2046294600F0E1
S31508000760A9FB4FF00A0744464FF002064FF0FF0870
S315080007704FF001052046314600F004FC0028F9D068
S315080007802046414600F0E8FB2046294600F0FAFBE1
S315080007900028F9D0013FEDD14FF40043ADF80430FD
S315080007A04FF003038DF806304FF018038DF8073025
S315080007B06C4C204601A900F023FB20464FF48051DB
S315080007C000F07AFB4FF000000146FFF7EDFE012826
S315080007D040F0BF8003F01AFC00F57A754FF0080068
S315080007E04FF4D571FFF7E0FE012849D10DF11B063C
S315080007F00DF11F0734464FF0FF084046FFF714FE79
S3150800080004F8010FBC42F8D19DF81E30012B40F0C8
S31508000810A0809DF81F30AA2B40F09B804FF0A908B6
S315080008204FF0804403F0F2FB854205D94046214645
S31508000830FFF7BAFE0028F5D103F0E8FB854240F23F
S3150800084088804FF03A004FF00001FFF7ADFE002810
S315080008507FD14FF0FF042046FFF7E6FD06F8010FAB
S31508000860BE42F8D19DF81C2002F04002D2B2002AFE
S3150800087014BF0C2204223C4B1A60FFF76FFE28E0D7
S315080008804FF0A9004FF00001FFF78EFE012899BF2F
S315080008900227A92401273C464FF0000603F0B6FBC1
S315080008A0854205D920463146FFF77EFE0028F5D158
S315080008B003F0ACFB85424CD94FF010004FF40071A1
S315080008C0FFF772FE002844D1274B1F60FFF746FE4C
S315080008D0A7B3234B1A7802F0FE021A70234D284656
S315080008E04FF0000100F028FB4FF00004ADF8084077
S315080008F04FF48273ADF80A30ADF80C40ADF80E40EF
S31508000900ADF810404FF40073ADF812304FF00803FD
S31508000910ADF81430ADF816404FF00703ADF81830AF
S31508000920284602A900F0E6FA2846214600F01AFBF6
S3150800093028464FF0010100F0FFFA04E0084B1A7848
S3150800094042F001021A70064B187811E04FF00100C8
S315080009500EE04FF00002044B1A60FFF7FFFDEDE7CB
S3150800096000000020000C0140300200200038004042
S3150800097009B0BDE8F08300BF10B9034B187870477B
S315080009804FF00100704700BF0000002070B50D460B
S315080009901C4600283ED1002B3FD0234B1B7813F072
S315080009A0010F3DD1214B1B6813F0080F08BF5202F7
S315080009B0012C0FD14FF011001146FFF7F5FD18BBBA
S315080009C028464FF40071FFF763FDD0F1010438BFE4
S315080009D0002419E04FF012001146FFF7E5FD98B91B
S315080009E04FF4007628463146FFF752FD30B105F53B
S315080009F0007504F1FF3414F0FF04F3D14FF00C0036
S31508000A004FF00001FFF7D0FDFFF7A8FD201C18BF27
S31508000A10012070BD4FF0040070BD4FF0040070BD9A
S31508000A204FF0030070BD00BF000000203002002018
S31508000A3070B50D4616461C46002850D1002B51D0DD
S31508000A402D4B1B7813F0010F4FD12B4B1B7803F05E
S31508000A500403DBB2002B4BD1284B1B6813F0080F9D
S31508000A6008BF5602012C0FD14FF018003146FFF788
S31508000A709BFD70BB28464FF0FE01FFF73BFDD0F10A
S31508000A80010438BF002424E013F0060F04D04FF009
S31508000A9097002146FFF788FD4FF019003146FFF70A
S31508000AA083FDB0B94FF0FC0628463146FFF722FD14
S31508000AB030B105F5007504F1FF3414F0FF04F3D1E5
S31508000AC04FF000004FF0FD01FFF714FD002808BFA6
S31508000AD00124FFF743FD201C18BF012070BD4FF00D
S31508000AE0040070BD4FF0040070BD4FF0030070BDE8
S31508000AF04FF0020070BD00BF000000203002002049
S31508000B0070B584B01446002840F06A81B84B1B784B
S31508000B1013F0010F40F067810E2900F23B81DFE8F0
S31508000B2011F00F0016003901680039013901390141
S31508000B30390139013901DE00E400F60008011F0118
S31508000B40FFF71AFDD0F1010438BF002445E14FF044
S31508000B5009004FF00001FFF727FD002840F01D812E
S31508000B6068464FF01001FFF793FC002800F0188143
S31508000B709DF800304FEA9313012B14D19DF80720F6
S31508000B8002F03F024FEA024202F101029DF80930E3
S31508000B909DF8081003EB0123D3184FEA832323603B
S31508000BA04FF0000419E19DF808209DF807304FEA38
S31508000BB0830303EB92139DF8062002F0030203EB6E
S31508000BC0822202F101029DF8053003F00F039DF819
S31508000BD00A1003EBD1139DF8091001F0030103EB8A
S31508000BE04103A3F1070302FA03F323604FF000045D
S31508000BF0F3E0804B1B6813F0040F2CD04FF08D00E8
S31508000C004FF00001FFF7D0FC002840F0CC804FF0F1
S31508000C10FF00FFF709FC68464FF01001FFF738FCA4
S31508000C20002800F0C3804FF030054FF0FF0630462D
S31508000C30FFF7FAFB05F1FF3313F0FF05F7D19DF82F
S31508000C400A304FEA13134FF0100202FA03F3236037
S31508000C504FF00004C1E04FF009004FF00001FFF724
S31508000C60A3FC002840F0A58068464FF01001FFF766
S31508000C700FFC002800F0A0805E4B1B6813F0020FE3
S31508000C8017D09DF80A2002F03F029DF80B304FEA74
S31508000C90D31303EB420202F101029DF80D304FEA2D
S31508000CA0931303F1FF3302FA03F323604FF00004B2
S31508000CB093E09DF80B309DF80A20C2F3840202F1F6
S31508000CC0010203F003014FEA531303EBC10303F1D7
S31508000CD0010303FB02F323604FF000047DE0454B5C
S31508000CE01B6813704FF0000477E04FF009004FF0CF
S31508000CF00001FFF759FC002861D120464FF010018A
S31508000D00FFF7C6FBD0F1010438BF002465E04FF0B9
S31508000D100A004FF00001FFF747FC002852D1204691
S31508000D204FF01001FFF7B4FBD0F1010438BF0024DF
S31508000D3053E04FF03A004FF00001FFF735FC00286A
S31508000D4043D14FF000054FF0FF063046FFF76CFB26
S31508000D50605505F10105042DF7D14FF000043CE07C
S31508000D60244B1B6813F0040F32D04FF08D004FF060
S31508000D700001FFF719FC70BB4FF0FF00FFF754FBAB
S31508000D8020464FF04001FFF783FBD0F1010438BF3E
S31508000D90002422E04FF004041FE04FF001041CE099
S31508000DA04FF0010419E04FF0010416E04FF001047A
S31508000DB013E04FF0010410E04FF001040DE04FF08E
S31508000DC001040AE04FF0010407E04FF0010404E0D3
S31508000DD04FF0010401E04FF00104FFF7BFFB04E008
S31508000DE04FF0040401E04FF00304204604B070BD40
S31508000DF00000002030020020004870470000AA4288
S31508000E002DE9F001CB7803F00F0513F0100F1CBF86
S31508000E108B781D430B7813B307684FF000034FF028
S31508000E2001064FF00F0C06FA03F20C8814409442A0
S31508000E3010D14FEA83020CFA02F827EA080705FAE6
S31508000E4002F21743CA78282A01D1446102E0482AE7
S31508000E5008BF046103F10103082BE4D107600B887E
S31508000E60FF2B24D947684FF000034FF001064FF0D7
S31508000E700F0C03F1080206FA02F20C881440944299
S31508000E8010D14FEA83020CFA02F827EA080705FA96
S31508000E9002F21743CA78282A08BF4461CA78482A42
S31508000EA008BF046103F10103082BE2D14760BDE8DE
S31508000EB0F0017047016170474161704721B1054BE8
S31508000EC09A69104398617047024B9A6922EA0000B2
S31508000ED0986170470010024021B1054BDA6910434A
S31508000EE0D8617047024BDA6922EA0000D861704778
S31508000EF00010024010B4028802F441524C880B8854
S31508000F0023438C882343CC8823430C8923434C8969
S31508000F1023438C892343CC89234313439BB2038001
S31508000F20838B23F400634FEA03434FEA1343838317
S31508000F300B8A038210BC704729B103889BB243F021
S31508000F40400303807047038823F040034FEA0343B6
S31508000F504FEA13430380704781817047808980B2C6
S31508000F60704700BF29B103889BB243F4005303803E
S31508000F707047038823F400534FEA03434FEA1343A9
S31508000F8003807047038919420CBF0020012070476F
S31508000F904FEAC1514FEAD1518180704703881942FF
S31508000FA00CBF00200120704742B101F1FF318218C1
S31508000FB011F8013F00F8013B9042F9D1704700BF94
S31508000FC022B1821800F8011B9042FBD1704700BF7E
S31508000FD0037833B18B4204D010F8013F0BB18B4232
S31508000FE0FAD11846704700BFCA7E8B7E43EA0223B1
S31508000FF00278032A05D1487D0A7D42EA002243EA9F
S3150800100002431846704700BF8176C1F30723C376AB
S315080010104FEA114101754FEA11214175704700BF2A
S3150800102000F10B014FF000034FEA530242EAC313E3
S3150800103010F8012B9B1803F0FF038842F4D11846D9
S31508001040704700BF08B588B1036893B1197899B19C
S31508001050D9888288914212D15878FFF78DFC00F022
S315080010600100002814BF0320002008BD4FF0090026
S3150800107008BD4FF0090008BD4FF0090008BD4FF044
S31508001080090008BD10B504460A46407804F1340143
S315080010904FF00103FFF77AFC98BB94F8332294F8D3
S315080010A0323243EA022212B21A4B9A422CD194F8EF
S315080010B06D2094F86C304FEA034343EA026294F8D1
S315080010C06A30134394F86B2043EA022222F07F42E7
S315080010D0114B9A421BD094F8890094F888304FEA4D
S315080010E0034343EA006094F88630034394F8870084
S315080010F043EA002020F07F40074BC01A18BF0120A2
S3150800110010BD4FF0030010BD4FF0020010BD4FF0A8
S31508001110000010BD55AAFFFF464154002DE9F041D5
S31508001120154603681C78A4F13004092C00F2DE8108
S315080011305A783A2A40F0DA8103F1020303604FF045
S3150800114000030B60002C40F07A81C74B1C68002C0A
S3150800115000F079810C6023788BB16078FFF70CFC7E
S3150800116010F0010F0BD1002D00F0718100F0040082
S31508001170C0B2002814BF0A200020BDE8F0814FF055
S31508001180000020706070FFF763FA10F0010F40F05E
S3150800119062812DB100F00400C0B2002840F05F81E2
S315080011A020464FF00001FFF76DFF012818D194F88B
S315080011B0F631002B00F0628194F8FD2194F8FC3199
S315080011C04FEA034343EA026294F8FA31134394F868
S315080011D0FB5143EA052520462946FFF753FF01E060
S315080011E04FF00005032800F04D81002840F04E819D
S315080011F094F8402094F83F3043EA02231BB2B3F533
S31508001200007F40F0478194F84B1094F84A3053EA2F
S3150800121001210ED194F85B2094F85A304FEA034323
S3150800122043EA026294F85830134394F8591043EA93
S315080012300121E16194F84420E27002F1FF33DBB248
S31508001240012B00F22B8194F84130A370002B00F09B
S31508001250298103F1FF30184240F0288194F846604E
S3150800126094F8450040EA0626B0B2208116F00F0F22
S3150800127040F0208194F8487094F8476056EA0726AB
S315080012800ED194F8577094F856604FEA064646EA27
S31508001290076794F854603E4394F8557046EA072663
S315080012A094F843C094F8427057EA0C2700F0068178
S315080012B002FB01FC07EB101262449642C0F0028161
S315080012C0B61AB6FBF3F3002B00F0008140F6F5766C
S315080012D0B3428CBF022601264FF6F578434500F245
S315080012E0098103F10203A3612562EF1967625219A6
S315080012F0E262032E15D1002840F0EC8094F86300D2
S3150800130094F862204FEA024242EA006094F86020AC
S31508001310024394F8610042EA0022A2624FEA83037C
S3150800132011E0002800F0DA806744A762022E02D195
S315080013304FEA430307E04FF0030202FB03F203F010
S31508001340010303EB520303F2FF13B1EB532FC0F073
S31508001350C9804FF0FF3323614FF00003E360032E8B
S315080013605FD1637194F8652094F8643043EA0222E9
S31508001370AA186261607804F134014FF00103FFF79F
S3150800138005FB00284DD194F8332294F8323243EA0B
S31508001390022212B2354B9A4243D194F8372094F878
S315080013A036304FEA034343EA026294F83430134373
S315080013B094F8352043EA02222D4B9A4231D194F80B
S315080013C01B2294F81A324FEA034343EA026294F85E
S315080013D01832134394F8192243EA0222254B9A42FB
S315080013E01FD194F8232294F822324FEA034343EAA2
S315080013F0026294F82032134394F8212243EA022326
S31508001400E36094F81F2294F81E324FEA034343EA36
S31508001410026294F81C32134394F81D2243EA02230D
S3150800142023612670144A138803F101039BB21380C3
S31508001430E3804FF0000020632071BDE8F0814FF093
S315080014400B00BDE8F0814FF00C00BDE8F0814FF0CD
S315080014500000BDE8F0814FF00300BDE8F0814FF0D1
S315080014600A00BDE8F08100BF3804002055AAFFFF36
S315080014705252614172724161340400204FF00D00EE
S31508001480BDE8F0814FF00100BDE8F0814FF00D0096
S31508001490BDE8F0814FF00D00BDE8F0814FF00D007A
S315080014A0BDE8F0814FF00D00BDE8F0814FF00D006A
S315080014B0BDE8F0814FF00D00BDE8F0814FF00D005A
S315080014C0BDE8F0814FF00D00BDE8F0814FF00D004A
S315080014D0BDE8F0814FF00D00BDE8F0814FF00D003A
S315080014E0BDE8F0814FF00D00BDE8F0814FF0000334
S315080014F00B602AE603F10203A3612562EF1967620E
S315080015005219E2624FF00306F5E600BF2DE9F041F5
S315080015100D4601F109040369002B60D0416991F871
S315080015200C800B78202B1BD00E46224604F1080CA3
S3150800153008F00807FFB203E016F8013F202B0FD08A
S31508001540052B08BFE52337B1A3F14104E4B2192CF2
S315080015509CBF2033DBB202F8013B14466245EBD14F
S315080015600B7A202B23D023464FF02E0203F8012BAB
S315080015700A7A202A1AD001F1080604F1040C08F0A8
S3150800158010085FFA88F703E016F8012F202A0ED014
S3150800159037B1A2F14104E4B2192C9CBF2032D2B271
S315080015A003F8012B1C466345EED100E01C46CB7AB6
S315080015B02B72CA7F8B7F4FEA034343EA02630A7F93
S315080015C013434A7F43EA02232B604A7E0B7E43EA93
S315080015D00223AB80CA7D8B7D43EA0223EB804FF062
S315080015E000032370AE6986B3EB6973B30369DBB195
S315080015F0028C4FF6FF739A4219D0C7693888C8B16A
S315080016004FF00004A046414601F080FDA8B1EA6902
S3150800161002F1FF32A24213D9305504F1010437F81A
S31508001620020F0028EFD10DE04FF000040AE04FF05A
S31508001630000407E04FF0000404E04FF0000401E066
S315080016404FF000044FF000033355BDE8F08100BFAA
S315080016502DE9F041044603794BB3056B00F13407D5
S31508001660407839462A464FF00103FFF7E1F910BBE7
S315080016704FF000032371636A9D4220D3E2699B18E9
S315080016809D4220D2E678012E21D94FF00108E26961
S31508001690AD18607839462A464346FFF7C9F906F178
S315080016A0FF36012EF3D14FF00000BDE8F0814FF070
S315080016B00000BDE8F0814FF00100BDE8F0814FF071
S315080016C00000BDE8F0814FF00000BDE8F0814FF062
S315080016D00000BDE8F08100BF38B504460D46036B2F
S315080016E08B420DD0FFF7B4FF68B9607804F1340176
S315080016F02A464FF00103FFF749F938B9256338BD83
S315080017004FF0000038BD4FF0010038BD4FF0010022
S3150800171038BD00BF70B50446FFF79AFF0346002898
S315080017205FD12378032B53D16379002B50D04FF028
S315080017300005256304F13406304629464FF4007245
S31508001740FFF73EFC4FF0550384F832324FF0AA03F8
S3150800175084F833324FF0520384F8343084F8353045
S315080017604FF0610384F836304FF0410284F8372091
S315080017704FF0720184F8181284F8191284F81A22A4
S3150800178084F81B32236984F81C32C3F3072284F8D1
S315080017901D224FEA134284F81E224FEA136384F887
S315080017A01F32E36884F82032C3F3072284F8212223
S315080017B04FEA134284F822224FEA136384F823324D
S315080017C06078314662694FF00103FFF731F96571B8
S315080017D060784FF000010A46FFF792F9031C18BF1C
S315080017E00123184670BD00BFA1F102018369A3F168
S315080017F00203994204D28278C36A02FB0130704719
S315080018004FF00000704700BFF8B505460C460129A1
S315080018106AD9836999426AD20378022B31D0032B9D
S3150800182043D0012B66D101EB5106416A01EB5621E3
S31508001830FFF752FF002860D14FEAC6534FEAD35349
S31508001840EB1893F8347006F10106696A284601EB2D
S315080018505621FFF741FF002852D14FEAC6564FEAF4
S31508001860D656AD1995F8340047EA002014F0010F52
S3150800187002D04FEA1010F8BD4FEA00504FEA105058
S31508001880F8BD416A01EB1421FFF726FF00283AD17B
S315080018904FEA04644FEAD4542B1993F834302C19C0
S315080018A094F8350043EA0020F8BD416A01EBD411EB
S315080018B0FFF712FF002829D14FEA44644FEAD454AF
S315080018C02B1993F8360093F837204FEA026242EA5A
S315080018D0004293F8350042EA00202C1994F8343077
S315080018E0184320F07040F8BD4FF00100F8BD4FF0E6
S315080018F00100F8BD4FF0FF30F8BD4FF0FF30F8BDDE
S315080019004FF0FF30F8BD4FF0FF30F8BD4FF0FF3015
S31508001910F8BD00BF70B504460D46E180816801290F
S315080019203CD003689A6991423BD279B91A78032A5E
S3150800193001D1996A51B94FF00002E2601A89AA42A8
S3150800194032D99B6A03EB151323611CE09E784FEA94
S315080019500616B54210D32068FFF756FF0146B0F1C8
S31508001960FF3F24D0012825D923689B69984224D2B1
S31508001970AD1BADB2AE42EED9E1602068FFF734FF89
S3150800198000EB1510206105F00F05236803EB4513DE
S3150800199003F1340363614FF0000070BD4FF002009D
S315080019A070BD4FF0020070BD4FF0020070BD4FF0E1
S315080019B0010070BD4FF0020070BD4FF0020070BD0F
S315080019C0F8B505460C461646012940F28980836912
S315080019D0994280F088800378022B44D0032B56D096
S315080019E0012B77D101EB5107416A01EB5721FFF72C
S315080019F073FE034600286FD14FEAC7534FEAD35305
S31508001A0014F0010409D0EA1892F8342002F00F0203
S31508001A10F1B242EA0112D2B200E0F2B2EB1883F850
S31508001A20342007F101074FF001032B71696A284634
S31508001A3001EB5721FFF750FE034600284CD14FEA29
S31508001A40C7574FEAD75714B1C6F3071607E0EA197E
S31508001A5092F8342022F00F02C6F303261643EF1934
S31508001A6087F8346038E0416A01EB1421FFF734FE49
S31508001A70034688BB4FEA04644FEAD4542A1982F80D
S31508001A8034601446C6F3072682F8356024E0416AB6
S31508001A9001EBD411FFF720FE0346E8B94FEA446488
S31508001AA04FEAD4542A1992F837104FEA01612C19D3
S31508001AB001F070410E4384F83460C6F3072182F8BA
S31508001AC035104FEA164182F836104FEA166682F844
S31508001AD0376001E04FF002034FF001022A7104E07B
S31508001AE04FF0020301E04FF002031846F8BD00BFAD
S31508001AF02DE9F0410546884631B9C66876B183694D
S31508001B009E4228BF01260BE0FFF77EFE034601280A
S31508001B1045D9AA6990424CD3464601E04FF00106E2
S31508001B2034464FF0020704F10104AB699C4202D324
S31508001B30012E37D93C4628462146FFF765FE03465F
S31508001B4038B1B0F1FF3F34D0012832D0B442EAD1DF
S31508001B502BE02646284621466FF07042FFF730FFF5
S31508001B600346B0B9B8F1000F06D0284641462246CA
S31508001B70FFF726FF034660B9EE602B69B3F1FF3F16
S31508001B8016D003F1FF332B614FF001036B71234627
S31508001B900FE0012B14BF01234FF0FF3309E04FF08C
S31508001BA0010306E04FF0000303E04FF0000300E0F6
S31508001BB023461846BDE8F0812DE9F84304460E464B
S31508001BC0C58805F10105ADB2002D70D00369002B5B
S31508001BD071D015F00F075FD103F101030361C168E6
S31508001BE021B903681B89AB4269D955E00068837837
S31508001BF003F1FF3313EA15134ED1FFF705FE8046AE
S31508001C00012860D9B0F1FF3F61D020688369984503
S31508001C103BD3002E5FD0E168FFF76AFF80460028B5
S31508001C205DD001285FD0B0F1FF3F60D02068FFF794
S31508001C300FFD00285FD1206800F134004FF0000145
S31508001C404FF40072FFF7BCF9266830464146FFF7A5
S31508001C50CBFD30634FF000064FF001090EE083F824
S31508001C6004902068FFF7F4FC002848D123681A6B13
S31508001C7002F101021A6306F10106F6B223689A78A0
S31508001C80B242ECD81A6B921B1A63C4F80C8020680F
S31508001C904146FFF7A9FD2061E580236803EB47135A
S31508001CA003F1340363614FF00000BDE8F8834FF099
S31508001CB00400BDE8F8834FF00400BDE8F8834FF050
S31508001CC00400BDE8F8834FF00200BDE8F8834FF042
S31508001CD00100BDE8F8834FF00400BDE8F8834FF033
S31508001CE00700BDE8F8834FF00200BDE8F8834FF01F
S31508001CF00100BDE8F8834FF00100BDE8F8834FF016
S31508001D000100BDE8F88300BF2DE9F04F87B004460F
S31508001D104FF00001FFF7FEFD0746002840F0C1809E
S31508001D204FF0FF09C846CA46604A02F10C02019202
S31508001D304FF0000B20682169FFF7CEFC0746002804
S31508001D4040F0AF8065692E78002E00F09980EB7A16
S31508001D5003F03F02E52E00F0838003F00803DBB2B0
S31508001D6013B10F2A7ED101E00F2A5AD1E769002F55
S31508001D707DD006F04003DBB233B195F80D9006F03E
S31508001D80BF06E388238403E0B04518BFD0466ED16A
S31508001D906B7B02934B4567D12B7823F0400303F105
S31508001DA0FF3303EB430203EB820203923F4A02F13D
S31508001DB0FF384FF001090596039E04944C46DDF85A
S31508001DC0049018F8013FEA185278EB5C43EA0220BF
S31508001DD074B101F0C1F90446FE2E5BD837F8160037
S31508001DE006F1010601F0B8F9844205D0049C54E0D6
S31508001DF04FF6FF7398424FD1C845E2D1A1460396E4
S31508001E00059E049C2B7803F04003DBB2002B3AD0E6
S31508001E10B9F1000F37D0039A37F81230002B32D0B9
S31508001E203BE0B8F1000F04D12846FFF7F9F848451A
S31508001E3037D04FF0FF332384A369DA7A12F0010F03
S31508001E4014D105F1FF3503F10B0001E0834228D0D8
S31508001E5013F8012B15F8011F9142F7D0D04606E07A
S31508001E60D04604E0D04602E0D04600E0D046204600
S31508001E705946FFF7A1FE074600283FF45BAF10E07E
S31508001E804FF004070DE006F1FF365FFA86F8DDF835
S31508001E900890ECE7049C00E0049CDDF80890D04626
S31508001EA0E5E7384607B0BDE8F08F00BF40460008B2
S31508001EB02DE9F04F85B0824688460B782F2B01D046
S31508001EC05C2B01D108F101084FF00003CAF808306D
S31508001ED098F800301F2B0AD850464FF00001FFF73C
S31508001EE019FD02464FF00003CAF814306FE14FF0AF
S31508001EF0010B454618F8013B2F2BFAD05C2BF8D07E
S31508001F00DAF81C6028781F2840F241812F2800F053
S31508001F1033815C2800F03481A6F102092F465C461D
S31508001F200AE02F2B00F02F815C2B00F02C81B8F5EE
S31508001F30807F00F041814446594601F0E7F8804623
S31508001F40002800F039817F2806D8A3484146FFF7C4
S31508001F503FF8002840F0308129F8028F17F8013F32
S31508001F60184604F101081F2BDBD813E1002C00F0FA
S31508001F70238106EB440232F8023D202B01D02E2B9A
S31508001F8002D1013CF7D117E1A146002C00F01481DB
S31508001F9006EB440101914FF0000226F81420DAF806
S31508001FA018004FF020014FF00B02FFF709F8A6F1D1
S31508001FB002024FF0000501E005F1010532F8023F83
S31508001FC0202BF9D02E2BF7D0002D00F0E78047F014
S31508001FD00307E3E0013C08D14FF0080301934FF0F3
S31508001FE0000102910391A14606E0A3F1020333F82A
S31508001FF0022C2E2AEED1EFE736F8154005F1010539
S31508002000002C63D0202C04D02E2C05D1A94500F035
S31508002010D68047F00307EFE7029B01998B4202D26D
S31508002020A9451AD1C3E0019A0B2A03D147F0030741
S3150800203003994EE0A94503D047F003074D4547D815
S3150800204003994FEA8103DBB203934D464FF00B0227
S3150800205001924FF008030293CEE77F2C0ED9204653
S315080020604FF0000101F052F8002800F0AD805B49FE
S315080020700B1813F8804C47F0020724B1584821463C
S31508002080FEF7A6FF20B147F003074FF05F0415E0FF
S31508002090A4F141039BB2192B04D8039A42F0020219
S315080020A003920BE0A4F161039BB2192B06D8039B9C
S315080020B043F001030393A4F12004A4B2DAF818301C
S315080020C002995C5401F10101029195E7039900E038
S315080020D00399DAF818301A78E52A04BF05221A7027
S315080020E0019A082A03D14FEA8101C9B203910399DB
S315080020F001F00C030C2B03D001F00302032A01D1D3
S3150800210047F0020707F00202D2B252B9039901F06A
S315080021100302012A08BF47F01007042B08BF47F03F
S315080021200807DAF81830DF725046FFF7EDFDDAF8DF
S315080021301830DB7A024648B1042848D103F0040374
S31508002140DAB2002A14BF0246052240E003F004036F
S31508002150DBB2002B3BD1DAF81410CB7A03F010036C
S31508002160DBB233B1DAF80000FEF73EFFCAF8080022
S31508002170BFE64FF005022AE04FF00004D84602E019
S315080021804FF00004D846A8444FF00007EEE64FF09B
S315080021900004D846A8444FF00407E7E609F1FF39DA
S315080021A036F819302E2B3FF417AF019B12E7019A28
S315080021B00B2A7FF445AF39E74FF0060207E0019B8B
S315080021C00B2B7FF43DAF31E747F002075BE710467C
S315080021D005B0BDE8F08F00BFAC450008C045000853
S315080021E0B84500082DE9F0410446C588018C4FF62C
S315080021F0FF73994208BF2946FFF78CFB0346E0B9EF
S315080022004FF0E5074FF001064FF0000820682169F6
S31508002210FFF762FA034668B9626917702268167191
S31508002220E288AA4209D220464146FFF7C5FC034682
S315080022300028EBD0042B08BF02231846BDE8F0811E
S315080022402DE9F04F83B0044689464FF0FF0A5646FB
S315080022504FF00405D046DFF828B10BF10C000090CA
S315080022604FF0000775E02068FFF736FA05460028A4
S3150800227073D162691378002B7BD0D17AE52B5BD0BA
S315080022802E2B5BD001F03F01082914BF0020012046
S31508002290484555D10F2945D103F04001C9B231B19E
S315080022A092F80DA003F0BF03E188218403E09E4263
S315080022B018BF464647D192F80DE0D64542D1D4F824
S315080022C01CC0117801F03F0101F1FF3101EB410516
S315080022D001EB85050BF1FF314FF001060193DDF89F
S315080022E000A011F8013FD0184078D35C43EA0023D8
S315080022F03EB1FE2D3AD82CF8153005F101051E46DB
S3150800230003E04FF6FF70834230D15145E9D1019B76
S31508002310127802F04002D2B21AB3FE2D26D82CF853
S3150800232015701EE010461EB9FEF77AFE504523D0FA
S315080023304FF6FF7323841FE0464604E0464602E054
S31508002340464600E0464620463946FFF735FC054630
S3150800235018B92169002986D175B14FF000032361A8
S315080023600AE003F1FF33DEB2F246ECE7F2464646F0
S31508002370E9E74FF00405F0E7284603B0BDE8F08F1B
S31508002380404600082DE9F04104460E46012926D9A3
S315080023908369994226D24FF000074FF0010820467C
S315080023A03146FFF731FA0546F8B1012820D0B0F1D9
S315080023B0FF3F20D0204631463A46FFF701FB01464B
S315080023C0D8B92369B3F1FF3F04D003F101032361B0
S315080023D084F805802E46A369AB42E0D80DE04FF09D
S315080023E002010AE04FF0020107E04FF0000104E0A5
S315080023F04FF0020101E04FF001010846BDE8F08107
S3150800240070B582B0054616461C464FF00B02FEF71D
S31508002410CBFD052C0CD9A6F102024FEA540343EA78
S31508002420C43432F8023FE418A4B25388002BF4D11E
S315080024304FF0070204F00F0101F13003392B88BF72
S3150800244001F137030DF8023002F1FF322409F1D108
S3150800245010464FF07E0102ACA31803F8081C72B1AF
S315080024602B78202B0ED029464FF0000303F10103E9
S31508002470834209D011F8014F202CF7D104E04FF020
S31508002480000301E04FF000034FF02000072A06D8AA
S3150800249002ACA11811F8081C02F1010200E001467D
S315080024A0E95403F10103072BF0D902B070BD00BF50
S315080024B02DE9F04F87B004468769C66903A83946EF
S315080024C04FF00C02FEF770FD9DF8173013F0010F60
S315080024D022D04FF00003FB72E3614FF00105384646
S315080024E003A932462B46FFF78BFF2046FFF70CFC65
S315080024F0824638B905F10105ADB2642DEFD14FF02A
S31508002500070AF8E0642D00F0D780042840F0F3802D
S315080025109DF81730FB72E6619DF8173003F0020349
S31508002520DBB2C3B133884BB14FF0000303F10103AB
S315080025309BB236F81320002AF8D101E04FF00003C9
S3150800254003F119036E4F87FB03274FEAE373C3EBC7
S31508002550A707BFB201E04FF0010720464FF0000180
S31508002560FFF7D8F98246002840F0C5804FF00005ED
S31508002570A8464FF0010620682169FFF7ADF88246A4
S31508002580002840F0B88063691B78E52B00D023B992
S3150800259005F10105AF4201D191E045462046314695
S315080025A0FFF70AFB82460028E5D0A4E0E188C8EBDD
S315080025B00101204689B2FFF7ADF98246002840F0AE
S315080025C09A80A069FEF72CFD01904FF000094FF69E
S315080025D0FF754C4E4FF0FF0720682169FFF77CF81E
S315080025E08246002840F08780D4F81CA061695FFA0B
S315080025F088FB019B4B734FF00F02CA7281F80C904F
S3150800260081F81A9081F81B900BF1FF3303EB430016
S3150800261003EB80004FF001024B4602E02B4602F125
S315080026200102AB4253D03AF8103000F1010006EB34
S31508002630020E1EF801EC01F80E308E444FEA132CF8
S315080026408EF801C0002B4CD00C2AE8D9AB4202D038
S315080026503AF810301BB948F0400B5FFA8BFB81F84B
S3150800266000B023684FF001021A7120464946FFF769
S31508002670A3FA824600283ED108F1FF381FFA88F8E7
S31508002680B8F1000FA8D12FE060694FF000014FF0B4
S315080026902002FEF795FC6069A1694FF00B02FEF770
S315080026A083FC6369A269D27A02F018021A73236856
S315080026B04FF001021A711EE04FF0070A1BE007F1FE
S315080026C0FF371FFA87F8B8F1000F0DD06EE706EB53
S315080026D0020E1EF801EC01F80E708E448EF8017099
S315080026E0B2E70C2A9AD9B6E720682169FEF7F4FF03
S315080026F082460028C8D0504607B0BDE8F08F00BF14
S315080027004FECC44E4046000870B9094B1B6813B11C
S315080027104FF000021A7011B14FF000030B70044B12
S3150800272019604FF0000070474FF00B00704700BF6C
S31508002730380400202DE9F0438FB00191164605466E
S31508002740002800F0A2804FF00003036001A805A945
S3150800275002F01E02FEF7E2FC0446002840F0B480B0
S3150800276006F01F0802AB0B93594B0C9305A8019969
S31508002770FFF79EFB0A9F0346002840F08F80002F34
S3150800278040F0868088E05BB1042B40F0928005A873
S31508002790FFF78EFE48F008080A9F50B1044693E0FA
S315080027A0FB7A13F0110F7ED106F00406F6B2002E5E
S315080027B07CD108F00803DBB2002B41D0FEF71CFBE6
S315080027C0B873C0F30723FB734FEA10433B744FEA11
S315080027D0106078744FF00006FE723E777E77BE77FB
S315080027E0FE7705983946FEF7FFFB8146384631469F
S315080027F0FEF70AFC05984FF001020271B9F1000FC5
S315080028001ED0066B4946FFF7BDFD002853D1059833
S3150800281009F1FF33C3603146FEF75EFF03460DE05C
S31508002820FB7A03F01002D2B2002A46D106F002065D
S31508002830F6B22EB113F0010F42D101E0002B42D1BE
S3150800284008F00803DBB20BB148F02008059E336B8D
S31508002850EB612F6285F8068030463946FEF7C4FBE1
S315080028602861FA7FBB7F4FEA034343EA02633A7F54
S3150800287013437A7F43EA0223EB604FF00003AB6011
S31508002880AB612E60F388AB801EE04FF009041BE0B5
S3150800289016F01C0F84D1C3E74FF0060316F01C0F81
S315080028A07FF471AFCAE74FF007040DE04FF0080454
S315080028B00AE01C4608E0044606E04FF0040403E07C
S315080028C04FF0070400E01C4620460FB0BDE8F08331
S315080028D0340200202DE9F04F83B00446884691461D
S315080028E01E464FF000033360FEF7ACFB0746002890
S315080028F040F0CE80A37913F0800F40F0C48013F027
S31508002900010F00F0C380E568A368ED1AA94538BF32
S315080029104D46002D00F0BC8004F12403009301907D
S31508002920A2684FEAC2534FEAD353002B40F08D807A
S31508002930206890F802A00AF1FF3A0AEA522A1AF029
S31508002940FF0A19D10AB9206902E06169FEF75CFF3E
S31508002950012806D8A37963F07F03A3714FF0020715
S3150800296096E0B0F1FF3F06D1A37963F07F03A37128
S315080029704FF001078CE06061276838466169FEF709
S3150800298033FF814630B9A37963F07F03A3714FF013
S3150800299002077DE000EB0A095FEA552B29D0BB78D0
S315080029A00BEB0A029A4288BFCAEB030B78784146BA
S315080029B04A465FFA8BF3FDF7E9FF30B1A37963F076
S315080029C07F03A3714FF0010762E0A37903F0400388
S315080029D0DBB25BB1A369C9EB0300834506D908EBF3
S315080029E0402000994FF40072FEF7DEFA4FEA4B2BAF
S315080029F03CE0A2694A4526D0A37903F04003DBB23E
S31508002A008BB1787800994FF00103FEF711F830B1D1
S31508002A10A37963F07F03A3714FF0010738E0A37928
S31508002A2023F04003A3712368587800994A464FF06B
S31508002A300103FDF7ABFF30B1A37963F07F03A37100
S31508002A404FF0010724E0C4F81890A1684FEAC15175
S31508002A504FEAD151C1F5007B5D4538BFAB466118D9
S31508002A60404601F124015A46FEF79EFAD844A36867
S31508002A705B44A36033685B443360B5EB0B057FF4B6
S31508002A804FAF019F04E04FF0020701E04FF0070740
S31508002A90384603B0BDE8F08F2DE9F04F83B0044601
S31508002AA0884615461E464FF000033360FEF7CAFAFD
S31508002AB00746002840F0EC80A37913F0800F40F019
S31508002AC0E28003F00203DBB2002B00F0DF80E3684C
S31508002AD0DD4280F0CE80002D00F0CB8004F1240387
S31508002AE000930190A2684FEAC2534FEAD353002BD2
S31508002AF040F09C80206890F802B00BF1FF3B0BEA8F
S31508002B00522B1BF0FF0B24D142B923696BB94FF046
S31508002B100001FEF7EDFF0346206103E06169FEF759
S31508002B20E7FF0346002B00F0A380012B06D1A3790B
S31508002B3063F07F03A3714FF00207A9E0B3F1FF3FEB
S31508002B4006D1A37963F07F03A3714FF001079FE0D5
S31508002B506361A37903F04003DBB29BB1236858781D
S31508002B600099A2694FF00103FDF762FF30B1A3791E
S31508002B7063F07F03A3714FF0010789E0A37923F07F
S31508002B804003A371276838466169FEF72DFE814622
S31508002B9030B9A37963F07F03A3714FF0020777E09A
S31508002BA000EB0B095FEA552A28D0BB780AEB0B0223
S31508002BB09A4288BFCBEB030A787841464A465FFAC1
S31508002BC08AF3FDF735FF30B1A37963F07F03A3716C
S31508002BD04FF001075CE0A369C9EB03018A450AD9EE
S31508002BE0009808EB41214FF40072FEF7DDF9A3794E
S31508002BF023F04003A3714FEA4A2A2CE0A3694B4508
S31508002C0012D0A268E3689A420ED2787800994A46AA
S31508002C104FF00103FDF7BAFE30B1A37963F07F03E5
S31508002C20A3714FF0010733E0C4F81890A0684FEA83
S31508002C30C0504FEAD050C0F5007A554538BFAA466D
S31508002C40201800F1240041465246FEF7ADF9A37953
S31508002C5043F04003A371D044A3685344A360336888
S31508002C6053443360B5EB0A057FF43CAF019F00E09F
S31508002C70019FA368E268934288BFE360A37943F0A3
S31508002C802003A37104E04FF0020701E04FF00707A5
S31508002C90384603B0BDE8F08F38B50446FEF7D2F9DA
S31508002CA00346002850D1A27902F02001C9B20029B2
S31508002CB04AD002F04002D2B272B1214651F8243B02
S31508002CC05878A2694FF00103FDF7B2FE002839D102
S31508002CD0A37923F04003A3712068E169FEF7FCFCA1
S31508002CE0034688BB256AEB7A43F02003EB72E36858
S31508002CF02B77A3894FEA13236B77E389AB77E37BBB
S31508002D00EB7728462169FEF77FF9FEF775F8A8756F
S31508002D10C0F30723EB754FEA10432B764FEA106092
S31508002D2068764FF00003AB74EB74A37923F02003A5
S31508002D30A37123684FF001021A712068FEF7EAFCB6
S31508002D40034601E04FF00103184638BD10B50446A6
S31508002D50FFF7A2FF034610B94FF00002226018469B
S31508002D6010BD00BFF8B504460D46FEF76BF90746D9
S31508002D70002840F0D380A37913F0800F40F0CC8070
S31508002D80E268AA4205D203F00203DBB2002B08BFB1
S31508002D901546A2684FF00003A360002D00F0BE8020
S31508002DA0206886784FEA462682B102F1FF3205F19D
S31508002DB0FF31B1FBF6F1B2FBF6F3994206D3C6F141
S31508002DC000031A40A260AD1A616919E02169B1B918
S31508002DD0FEF78EFE0146012806D1A37963F07F032C
S31508002DE0A3714FF0020799E0B0F1FF3F06D1A3792E
S31508002DF063F07F03A3714FF001078FE020616161E3
S31508002E00002946D0B5422ED9A27902F00202D2B2E2
S31508002E102AB12068FEF76CFE014620B922E0206838
S31508002E20FEF7F2FC0146B1F1FF3F06D1A37963F044
S31508002E307F03A3714FF0010770E0012903D92268C7
S31508002E409269914206D3A37963F07F03A3714FF089
S31508002E50020763E06161A2689219A260AD1BAE42E7
S31508002E60D2D300E03546A2685219A2604FEAC5528D
S31508002E704FEAD25282B12068FEF7B6FC30B9A37980
S31508002E8063F07F03A3714FF0020747E000EB552577
S31508002E9004E04FF0000501E04FF00005A3684FEA93
S31508002EA0C3534FEAD3536BB3A269AA422AD0A37974
S31508002EB003F04003DBB29BB1214651F8243B587816
S31508002EC04FF00103FDF7B4FD30B1A37963F07F033A
S31508002ED0A3714FF0010721E0A37923F04003A37102
S31508002EE0214651F8243B58782A464FF00103FDF74E
S31508002EF04DFD30B1A37963F07F03A3714FF001074D
S31508002F000CE0A561A368E268934207D9E360A37958
S31508002F1043F02003A37101E04FF002073846F8BDDD
S31508002F2030B58FB00EAB43F8340D0D46184605A9DB
S31508002F304FF00002FEF7F2F8044690B902AB0B9385
S31508002F40094B0C9305A80199FEF7B2FF044640B950
S31508002F500A9B23B105A82946FEF7D8FA01E04FF0E7
S31508002F60060420460FB030BD3402002030B599B0B3
S31508002F7018AB43F85C0D18460FA94FF00102FEF78F
S31508002F80CDF80346002854D103AB15932A4B169364
S31508002F900FA80199FEF78CFF0346002849D114991A
S31508002FA059B3CC7A14F0010F2AD12CE0012D34D96B
S31508002FB006A80FA94FF02402FDF7F6FF089506A804
S31508002FC04FF00201FEF7A6FC0346002831D106A8F9
S31508002FD04FF00001FFF734F9034640B304281FD029
S31508002FE027E02DB10F982946FFF7CCF9034600BB19
S31508002FF00F98FEF78FFB03461BE04FF0060318E019
S315080030004FF0070315E00F98FDF7EEFF054604F0AD
S315080030101004E4B2002CC9D102E04FF0020308E024
S315080030200FA8FFF7DFF803460028DAD001E04FF0D3
S315080030300703184619B030BD340200202DE9F047C1
S3150800304082B08246914604464FF0000501F1FF37EB
S315080030504FF0010814E0484601A942466B46FFF7BF
S3150800306039FC009B012B0ED19DF804300D2B08D09E
S31508003070337004F10104264605F101050A2B02D036
S315080030802646AF42E7DC4FF0000333709D4214BF7B
S315080030905046184602B0BDE8F08700BF30B583B089
S315080030A004460D460A2803D14FF00D00FFF7F6FF38
S315080030B002A901F8084D284669464FF0010201ABFE
S315080030C0FFF7EAFC0198012814BF4FF0FF300120F2
S315080030D003B030BD70B505460E46007870B14FF0A6
S315080030E000043146FFF7DAFFB0F1FF3F09D004F1DB
S315080030F0010415F8010F0028F3D104E04FF000048D
S3150800310001E04FF0FF34204670BD00BF7F2820D96C
S3150800311011B9C72808D114E0FF2818D8A0F18000F3
S315080031200C4B33F8100070470A4A4FF0010332F887
S31508003130021F814207D003F101039BB2802BF6D10F
S3150800314001E04FF0000303F18000C0B270474FF072
S31508003150000070473048000861280BD008494FF036
S31508003160000202F1010231F8023F43B18342F8D16D
S3150800317013B970474FF00002024B33F8120070473C
S31508003180504600083049000808B500F05DFA00F01E
S3150800319017FF00F0F3FE00F0DFFB00F00FF800F079
S315080031A043FA08BD08B500F051FA00F01FFF00F019
S315080031B00DFC00F01DF800F015FA08BD00B583B047
S315080031C04FF0FF038DF804304FF000038DF80530FB
S315080031D000F044F800F04AFE044B1B78012B02D19C
S315080031E001A800F059F803B000BD00BF3C04002058
S315080031F008B5044800F082FE012802D1014800F013
S315080032004BF808BD40040020704700BF08B5C9B296
S3150800321000F042FE00F038F808BD00BF4FF001028A
S31508003220014B1A70704700BF3C04002008B500F037
S3150800323023F808BD4FF00002014B5A70704700BFD3
S3150800324080040020044B4FF0FE02DA7018714FF02C
S315080032500202A3F84420704780040020054B4FF073
S3150800326000021A709A6483F84320A3F844209A70DF
S315080032705A70704780040020024B1878003018BF37
S3150800328001207047800400204FF00002014B83F8AC
S31508003290432070478004002038B504460378FF2B86
S315080032A022D100F06FFB20B94FF01000FFF7CAFFDC
S315080032B081E1FFF7BFFFAF4B4FF001021A704FF0E5
S315080032C0FF01D9704FF0100119714FF000015971C3
S315080032D04FF040009871D87119725A729A724FF06D
S315080032E00802A3F8442066E1A24A1278012A40F0AF
S315080032F07681A3F1C903352B00F25981DFE813F073
S31508003300D300570157015201570157014701EE00F3
S315080033102E011B0157015701570157015701570144
S3150800332057015701570157015701570157015701CF
S3150800333057015701570157015701570157015701BF
S3150800334057015701570157015701570157015701AF
S31508003350570157017900510036006E005701570191
S3150800336057019B005701AF00B400C50042783F2AB9
S3150800337004D94FF02200FFF765FF1CE17D4D05F1EA
S315080033800400A96C00F028FD4FF0FF03EB7062788B
S31508003390AB6CD318AB64637803F10103A5F844302A
S315080033A009E143783F2B04D94FF02200FFF74AFF83
S315080033B001E141686F4DA96405F10400627800F0E7
S315080033C00BFD4FF0FF03EB706278AB6CD318AB6460
S315080033D0637803F10103A5F84430ECE0654B4FF040
S315080033E0FF02DA7042689A644FF00102A3F844209B
S315080033F0E1E0604B4FF0FF02DA709B6C406848B121
S31508003400C0184FF0000213F8011B5218D2B28342BB
S31508003410F9D101E04FF00002564BC3F807204FF0F0
S3150800342001021A714FF000025A719A714FF00802A0
S31508003430A3F84420BFE04F4B4FF0FF02DA704E4A24
S315080034409A644FF000021A715A719A714FF0070286
S31508003450C3F807204FF00802A3F84420ABE04FF06A
S315080034600000FFF7EFFEA6E0424B4FF0FF02DA70CE
S315080034704FF000021A71597859719A71DA711A72F5
S315080034804FF00602A3F8442095E03A4C4FF00003AB
S315080034902370FFF7CFFE4FF0FF03E3704FF00103F1
S315080034A0A4F8443087E0334B986C4FF03F0104F1A1
S315080034B0010200F067FD20B94FF03100FFF7C2FEA8
S315080034C079E02C4B4FF0FF02DA709A6C02F13F025A
S315080034D09A644FF00102A3F844206CE043783E2B2F
S315080034E004D94FF02200FFF7ADFE64E0214B4FF000
S315080034F0FF02DA704FF00102A3F84420417841B97F
S3150800350000F04CFD002856D14FF03100FFF79AFE27
S3150800351051E0184B986C04F1020200F033FD20B913
S315080035204FF03100FFF78EFE45E0124B61789A6C3A
S315080035308A189A643FE00F4B4FF0FF02DA704FF09B
S3150800354000021A715A714FF040019971DA711A72B4
S315080035505A724FF00702A3F844202CE0054B986CEA
S31508003560616800F013FD48B94FF03100FFF76AFEB5
S3150800357021E000BF80040020104B0008184B4FF0D4
S31508003580FF02DA704FF00102A3F8442013E000F0BE
S3150800359035FC134B4FF0FF02DA704FF00102A3F827
S315080035A0442008E04FF03100FFF74CFE03E04FF0EF
S315080035B02000FFF747FE0A4B93F84330012B03D14F
S315080035C04FF01000FFF73EFE054B4FF0010283F85F
S315080035D0432003F10300B3F84410FFF717FE38BD84
S315080035E08004002008B5FFF721FE012817D000F057
S315080035F0C9F9A0B10A4B1B78012B10D100F006FDC2
S31508003600084B1B6803F13203984208D34FF00002B7
S31508003610034B1A7000F0C0F908B900F0C9FB08BDE1
S31508003620CC040020D004002008B54FF00102044B5A
S315080036301A7000F0EBFC034B1860FFF7D3FF08BDC8
S31508003640CC040020D0040020704700BF704700BF9C
S3150800365000F00F03092802D903F13700704703F178
S315080036603000054B1B681B185B7803F00303022B1D
S3150800367008BF2038C0B270470400002038B5054698
S315080036800C464FEA1010FFF7E3FF207005F00F0015
S31508003690FFF7DEFF60704FF00003A370204638BDC9
S315080036A030B403460F4C01F10101A4FB0323DB08E8
S315080036B0F9D14FF0000301F801390246094D0846D1
S315080036C0A5FB02434FEAD30303EB8304A2EB4402B0
S315080036D002F1300201F801291A46002BEFD130BC5D
S315080036E0704700BFCDCCCCCC70B40646164B1D68CF
S315080036F04FF000031846F15C6A18527802F003028C
S31508003700022A08BF2039C9B2A1F13002D2B2162A5C
S3150800371012D8A1F13A04E4B2062C10D9092A84BFBA
S31508003720A1F13702D2B202EB001000F0FF0003F15C
S315080037300103022BDFD104E04FF0000001E04FF057
S31508003740000070BC704700BF040000202DE9F04F50
S3150800375083B080461746894601B120B97C484FF4A4
S31508003760157100F019FB98F800307A4A1268D118DA
S31508003770497801F00301022908BF203B532B40F08A
S31508003780C38098F80130D218527802F00402D2B2F7
S31508003790002A00F0BC80312B00F0C380322B00F0E9
S315080037A0C380332B00F0C3804FF00005B7E02046F6
S315080037B0FFF79AFF3018C6B205F1FF35ADB204F12E
S315080037C00204012DF3D82046FFF78EFF6FEA06069E
S315080037D0F6B2864240F09E80BAF1010F2FD0BAF1B8
S315080037E0000F04D0BAF1020F40F0978056E0584611
S315080037F0FFF77AFF4FEA0024C9F8004008F10600EF
S31508003800FFF772FF2018C9F8000008F10808019BA5
S31508003810A3F10305ADB2002F00F081802EB2002E71
S315080038207DDD4FF000044046FFF75EFF385508F18E
S31508003830020804F10104A4B2B442F4DB6FE058466E
S31508003840FFF752FF4FEA0044C9F8004008F10600A6
S31508003850FFF74AFF04EB0024C9F8004008F1080006
S31508003860FFF742FF2018C9F8000008F10A08019B73
S31508003870A3F10405ADB2002F51D02EB2002E4EDDB5
S315080038804FF000044046FFF72FFF385508F10208AD
S3150800389004F10104A4B2A642F4DC40E05846FFF75E
S315080038A023FF4FEA0064C9F8004008F10600FFF755
S315080038B01BFF04EB0044C9F8004008F10800FFF7B5
S315080038C013FF04EB0024C9F8004008F10A00FFF7CB
S315080038D00BFF2018C9F8000008F10C08019BA3F19A
S315080038E00505ADB2DFB12EB2002E18DD4FF000048B
S315080038F04046FFF7F9FE385508F1020804F10104BD
S31508003900A4B2B442F4DB0AE04FF0000507E04FF03A
S31508003910000504E04FF6FF7501E04FF0000528B2F8
S3150800392012E04FF0000A04E04FF0010A01E04FF000
S31508003930020A08F10200FFF7D7FE0646019008F1D1
S31508003940040B05465C4632E703B0BDE8F08F00BFBE
S31508003950184B00080400002008B54FF00000064B7D
S3150800396018700649FEF7D0FE20B105484FF09101C0
S3150800397000F012FA08BD00BF14050020200500203B
S31508003980184B0008034B1878D0F1010038BF002007
S31508003990704700BF1405002008B5FFF747FC01284B
S315080039A009D0094B1B784BB9FCF710FC012808D144
S315080039B0054B187008BD4FF0000008BD4FF0000019
S315080039C008BD4FF0000008BD1405002070B5964BE1
S315080039D01B78002B00F0C481012B2BD1FCF71EFCB1
S315080039E09248FCF759FC9248FCF756FCFCF712FC87
S315080039F0014690484FF00102FEF79CFE38B18E480A
S31508003A00FCF74AFC4FF00100FCF73AFC70BD8B4806
S31508003A10FCF742FC8A48FCF73FFC8A48FCF73CFC6A
S31508003A20894B4FF000021A605A604FF002027E4B33
S31508003A301A7070BD022B40F0BB80844D84484FF449
S31508003A40807105F50D72FFF7F9FA95F93A32002BF0
S31508003A500FDA7948FCF720FC4FF00200FCF710FC5F
S31508003A6005F50D70FFF772F94FF000026E4B1A70EC
S31508003A7070BDD0B17649084601F5C0714FF0000215
S31508003A80FFF764FE0446B0F1FF3F0ED16A48FCF723
S31508003A9003FC4FF00300FCF7F3FB6648FFF756F903
S31508003AA04FF00002604B1A7070BD23B2002B17DD71
S31508003AB0654B5B683BB9644B654AD2F880211A604E
S31508003AC024B25C600CE0624AD2F880215E4909683B
S31508003AD08A423CBF5C490A6024B2E3185A4A5360DA
S31508003AE05A4BD3F83C22D3F840329A4240F03881F8
S31508003AF050484FF00001FFF735F970B14E48FCF712
S31508003B00CBFB4FF00400FCF7BBFB4A48FFF71EF956
S31508003B104FF00002444B1A7070BD4848FCF7BCFBD6
S31508003B204C48FCF7B9FB484D4B4C68682146FFF7F3
S31508003B30B7FD2046FCF7B0FB4848FCF7ADFB2E68FE
S31508003B404FEA16602146FFF799FDC6F3074004F1D0
S31508003B500201FFF793FDC6F3072004F10401FFF7FE
S31508003B608DFDF0B204F10601FFF788FD2046FCF74B
S31508003B7093FB3B48FCF790FB2868696800F006FA57
S31508003B8070B92D48FCF788FB4FF00500FCF778FB69
S31508003B902848FFF7DBF84FF00002234B1A7070BD78
S31508003BA02648FCF779FB4FF003021F4B1A7070BDCD
S31508003BB0032B40F0D580254D25484FF4807105F537
S31508003BC00D72FFF73BFA95F93A32002B0FDA2548C2
S31508003BD0FCF762FB4FF00200FCF752FB05F50D708F
S31508003BE0FFF7B4F84FF000020F4B1A7070BD0028AB
S31508003BF03CD0174A104602F5C07102F58072FFF7ED
S31508003C00A5FD0446B0F1FF3F30D11748FCF744FB49
S31508003C104FF00300FCF734FB0648FFF797F84FF020
S31508003C200002014B1A7070BD14050020304B0008C5
S31508003C30544B0008540700207C4B0008844B0008AE
S31508003C408C4B0008B04B0008180500202005002002
S31508003C5078090020E04B0008D4040020EC4B00084B
S31508003C60904C0008084C00082C4C000823B2002B86
S31508003C7046DD3C48FCF710FB24B23B4D204629465E
S31508003C80FFF70EFD2846FCF707FB3848FCF704FB50
S31508003C90374E96F883012946FFF7F0FC96F882011D
S31508003CA005F10201FFF7EAFC96F8810105F1040126
S31508003CB0FFF7E4FC96F8800105F10601FFF7DEFC44
S31508003CC02846FCF7E9FA2B48FCF7E6FAD6F880010D
S31508003CD0214606F5807200F055F970B92648FCF7BA
S31508003CE0DBFA4FF00600FCF7CBFA2448FFF72EF86C
S31508003CF04FF00002224B1A7070BD2248FCF7CCFA2E
S31508003D00214BD3F83C22D3F840329A4228D11F4897
S31508003D10FCF7C2FA00F042F970B91748FCF7BCFA8A
S31508003D204FF00700FCF7ACFA1448FFF70FF84FF00E
S31508003D300002134B1A7070BD1248FCF7ADFA14480E
S31508003D40FCF7AAFA0D48FFF701F81248FCF7A4FA9F
S31508003D504FF000020A4B1A70FCF776FA00F028F8C2
S31508003D6070BD00BF504C0008D4040020604C000809
S31508003D7078090020904C00087C4B00085407002066
S31508003D8014050020844B000820050020784C000804
S31508003D90944C0008AC4C000808B5034B1860034B5C
S31508003DA01960FFF753FCFCE7FC0A0020000B002013
S31508003DB008B500F0EFF850B1FFF726FA00F0F8F86A
S31508003DC04FF4C042024B1A60024B1B68984708BD65
S31508003DD008ED00E00460000870B5044602F1FF36FD
S31508003DE0B6B252B100F101039E190D1A635D04F8CB
S31508003DF0013BFFF72BFCB442F8D170BD08B500F0C3
S31508003E0087FB08BD074B1B8803F020039BB22BB129
S31508003E10044B9B8803704FF0010070474FF0000079
S31508003E20704700BF0044004010B50F4B1B8803F0D5
S31508003E3080039BB293B10C4B98801B8803F08003D8
S31508003E409BB273B9084CFFF701FC238803F0800383
S31508003E509BB2002BF7D04FF0010010BD4FF00000C9
S31508003E6010BD4FF0010010BD00440040094B4FF053
S31508003E7000021A819A811A829A821A8340F2712262
S31508003E801A819A8992B242F4005242F00C029A813F
S31508003E90704700BF004400402DE9F04106460C4635
S31508003EA0402904D914484FF08801FFF775FF2046CA
S31508003EB0FFF7BAFF012804D00F484FF08B01FFF730
S31508003EC06BFF2546ACB14FF00004DFF82C804FF0AD
S31508003ED09307FFF7BBFB305DFFF7A6FF012803D06A
S31508003EE040463946FFF758FF04F10104A3B2AB4236
S31508003EF0EFD3BDE8F08100BFD84C000838B50546B9
S31508003F001A4B1B786BB91A48FFF77CFF012824D196
S31508003F104FF00102154B1A704FF00000154B187040
S31508003F2038BD144B1C7814482018FFF76BFF01287E
S31508003F3016D104F10104E2B20E4B1A700C4B1B7831
S31508003F40934210D128460C49FFF746FF4FF000026E
S31508003F50064B1A704FF0010038BD4FF0000038BD0F
S31508003F604FF0000038BD4FF0000038BD480B002068
S31508003F70040B0020490B0020050B002008B500F0B3
S31508003F8083F908BD08B500F08BF908BD08B500F03F
S31508003F90B1F908BD08B500F065FA08BD08B500F026
S31508003FA039FA10B100F08AFA08BD4FF0000008BDD2
S31508003FB04FF00002014B1A60704700BF10E000E0A6
S31508003FC008B5FFF7F5FF064B064A5A604FF00002A0
S31508003FD09A604FF005011960034B1A8008BD00BFAF
S31508003FE010E000E03F1901004A0B0020054B1B6852
S31508003FF013F4803F04D0044B1A8802F101021A8098
S31508004000704700BF10E000E04A0B002008B5FFF734
S31508004010EDFF014B188808BD4A0B0020044B054AE2
S315080040205A6002F188325A604FF03402DA607047FB
S315080040300020024023016745024B1A6942F08002BC
S315080040401A61704700200240F8B507464FF0000491
S3150800405025460D4EFFF7FAFAA359BB420BD831197C
S3150800406049685B189F4206D205EB4502064B03EBEF
S315080040708202107AF8BD05F1010504F10C049C2CA6
S31508004080E8D14FF0FF00F8BDFC4C00082DE9F041DF
S3150800409080460068FFF7D8FFFF2847D0FFF7BEFF26
S315080040A0254BDB6813F0010F04D0FFF7C5FF4FF06F
S315080040B000043DE0204B1A6942F001021A614FF0F4
S315080040C000051C46D8F80030EF1808EB05025668BC
S315080040D0B2B2EA52E36813F0010F05D0FFF7B6FA59
S315080040E0E36813F0010FF9D14FEA16437B80E368C2
S315080040F013F0010F05D0FFF7A9FAE36813F0010FD3
S31508004100F9D13B68B34207D105F10405B5F5007F3F
S31508004110D8D14FF0010401E04FF00004064B1A69AC
S3150800412022F001021A61FFF787FF01E04FF0000451
S315080041302046BDE8F08100BF0020024070B5064663
S315080041400B4D4FF00004FFF781FA2B7AB34205D1E5
S3150800415004EB4402064B53F8220070BD04F1010437
S3150800416005F10C050D2CEED14FF0FF3070BD00BFE8
S31508004170FC4C000808B54FEAC1534FEAD3535BB964
S3150800418003688B420BD040F8041B4FF40072FFF70C
S3150800419023FE4FF0010008BD4FF0000008BD4FF0A8
S315080041A0010008BD38B504460D460C4B984206D0AA
S315080041B00B4B994205D0FFF769FF18B90AE0094C7D
S315080041C000E0064C20462946FFF7D4FF002808BF22
S315080041D0002401E04FF00004204638BD4C0B0020B7
S315080041E000600008500D00202DE9F84306460C46ED
S315080041F015461F464FEA51294FEA49290268B2F186
S31508004200FF3F03D14946FFF7B5FF88B333684B45EF
S3150800421005D030464946FFF7C5FF064660B3336802
S31508004220E41A341904F1040407F1FF381FFA88F870
S3150800423008F10108A84440F2FF1709F50079FFF7CD
S3150800424005FA06F10403E31ABB4207D93046494684
S31508004250FFF7A8FF064698B100F1040415F8013BDC
S3150800426004F8013B4545EAD14FF00100BDE8F88363
S315080042704FF00000BDE8F8834FF00000BDE8F88372
S315080042804FF00000BDE8F8834FF0FF33024A136091
S31508004290024A1360704700BF500D00204C0B0020E7
S315080042A070B504460D461646FFF7CEFEFF2814D015
S315080042B004F1FF304019FFF7C7FEFF2810D04FEA78
S315080042C05422094BB3EB422F0CBF08480848214635
S315080042D03246ABB2FFF788FF70BD4FF0000070BDE5
S315080042E04FF0000070BD00BF006000084C0B0020B6
S315080042F0500D00202DE9F04106460C46FFF7A4FEB6
S31508004300054606F1FF300019FFF79EFE0446FF2D0D
S3150800431073D0FF2875D0854263D8022D65D90F283A
S3150800432067D8FFF77BFE394BDB6813F0010F05D022
S31508004330FFF782FE4FF00000BDE8F081334B1A69A3
S3150800434042F002021A612846FFF7F8FE07462046A1
S31508004350FFF7F4FE80462E4E4FF00005FFF776F97C
S31508004360337AA34206D105EB4502294B03EB8203B8
S315080043705B6807E005F1010506F10C060D2DEDD188
S315080043804FF00003C7EB08084344C3F38F23EBB190
S3150800439003F1FF339EB206F101064FEA86264FF077
S315080043A000051A4CEB196361236943F04003236146
S315080043B0E36813F0010F05D0FFF748F9E36813F037
S315080043C0010FF9D105F58065B542EBD10F4B1A6996
S315080043D022F002021A61FFF72FFE4FF00100BDE836
S315080043E0F0814FF00000BDE8F0814FF00000BDE815
S315080043F0F0814FF00000BDE8F0814FF00000BDE805
S31508004400F0814FF00000BDE8F08100BF00200240B7
S31508004410FC4C000800B583B0104B1B68B3F1FF3F96
S3150800442018D00E4B99685A688918DA6889181A6973
S3150800443089185A6989189A698A18D9695318C3F163
S31508004440000302AA42F8043D05484FF00401FFF7AD
S3150800445027FF01E04FF0010003B000BD4C0B002020
S31508004460506100080E4B1868A3F104031B68C018B6
S315080044700C4B1B68C0180C4B1B68C0180B4B1B68F1
S31508004480C0180B4B1B68C0180A4B1B68C0180A4B90
S315080044901B68C018D0F1010038BF0020704700BF64
S315080044A004600008086000080C6000081060000836
S315080044B014600008186000085061000808B50D4B24
S315080044C01B68B3F1FF3F03D00A48FFF7DFFD58B179
S315080044D0094B1B68B3F1FF3F09D00748FFF7D6FD24
S315080044E0003018BF012008BD4FF0000008BD4FF08E
S315080044F0010008BD4C0B0020500D002008B50348EC
S315080045004FF03601FFF748FC08BD00BF984D00087C
S3150800451010B572B6114B124A9A4211D202F104032F
S31508004520104CE41A24F0030404F104044FF00003C9
S3150800453010460D495A581A5003F10403A342F9D1FB
S315080045400A480B494FF000028842B8BF40F8042BCE
S31508004550FFF6FAAFFBF7CAFE10BD00BF0800002041
S31508004560000000200B000020C84E000808000020AC
S31508004570540F00202F64656D6F70726F675F6F6CE4
S31508004580696D65785F73746D3332703130332E73AD
S31508004590726563002F626F6F746C6F672E74787420
S315080045A0000000006D61696E2E630000222A3A3C05
S315080045B03E3F7C7F000000002B2C3B3D5B5D0000EE
S315080045C0809A90418E418F804545454949498E8F4D
S315080045D09092924F994F555559999A9B9C9D9E9F9B
S315080045E041494F55A5A5A6A7A8A9AAABAC21AEAF28
S315080045F0B0B1B2B3B4B5B6B7B8B9BABBBCBDBEBF35
S31508004600C0C1C2C3C4C5C6C7C8C9CACBCCCDCECF24
S31508004610D0D1D2D3D4D5D6D7D8D9DADBDCDDDEDF14
S31508004620E0E1E2E3E4E5E6E7E8E9EAEBECEDEEEF04
S31508004630F0F1F2F3F4F5F6F7F8F9FAFBFCFDFEFFF4
S3150800464001030507090E10121416181C1E00000097
S315080046506100620063006400650066006700680028
S3150800466069006A006B006C006D006E006F007000D8
S315080046707100720073007400750076007700780088
S3150800468079007A00A100A200A300A500AC00AF0043
S31508004690E000E100E200E300E400E500E600E700F0
S315080046A0E800E900EA00EB00EC00ED00EE00EF00A0
S315080046B0F000F100F200F300F400F500F600F8004F
S315080046C0F900FA00FB00FC00FD00FE00FF000101F6
S315080046D003010501070109010B010D010F01110174
S315080046E013011501170119011B011D011F012101E4
S315080046F023012501270129012B012D012F01310154
S315080047003301350137013A013C013E0140014201BE
S315080047104401460148014B014D014F015101530126
S315080047205501570159015B015D015F016101630193
S315080047306501670169016B016D016F017101730103
S31508004740750177017A017C017E019201B103B203FA
S31508004750B303B403B503B603B703B803B903BA037F
S31508004760BB03BC03BD03BE03BF03C003C103C3032E
S31508004770C403C503C603C703C803C903CA03300471
S315080047803104320433043404350436043704380457
S3150800479039043A043B043C043D043E043F04400407
S315080047A041044204430444044504460447044804B7
S315080047B049044A044B044C044D044E044F04510466
S315080047C0520453045404550456045704580459040F
S315080047D05A045B045C045E045F0470217121722133
S315080047E073217421752176217721782179217A21FF
S315080047F07B217C217D217E217F2141FF42FF43FFD2
S3150800480044FF45FF46FF47FF48FF49FF4AFF4BFF66
S315080048104CFF4DFF4EFF4FFF50FF51FF52FF53FF16
S3150800482054FF55FF56FF57FF58FF59FF5AFF000020
S31508004830C700FC00E900E200E400E000E500E7004C
S31508004840EA00EB00E800EF00EE00EC00C400C5004B
S31508004850C900E600C600F400F600F200FB00F90005
S31508004860FF00D600DC00A200A300A500A720920145
S31508004870E100ED00F300FA00F100D100AA00BA0049
S31508004880BF001023AC00BD00BC00A100AB00BB00FC
S3150800489091259225932502252425612562255625ED
S315080048A055256325512557255D255C255B2510254E
S315080048B0142534252C251C2500253C255E255F2539
S315080048C05A25542569256625602550256C256725B2
S315080048D068256425652559255825522553256B25B0
S315080048E06A2518250C25882584258C25902580255C
S315080048F0B103DF009303C003A303C303B500C403D6
S31508004900A6039803A903B4031E22C603B5032922E6
S315080049106122B1006522642220232123F700482260
S31508004920B0001922B7001A227F20B200A025A000E5
S315080049304100420043004400450046004700480045
S3150800494049004A004B004C004D004E004F005000F5
S3150800495051005200530054005500560057005800A5
S3150800496059005A002100E0FFE1FFE5FFE2FFE3FFFF
S31508004970C000C100C200C300C400C500C600C7000D
S31508004980C800C900CA00CB00CC00CD00CE00CF00BD
S31508004990D000D100D200D300D400D500D600D8006C
S315080049A0D900DA00DB00DC00DD00DE00780100015A
S315080049B002010401060108010A010C010E01100199
S315080049C012011401160118011A011C011E01200109
S315080049D022012401260128012A012C012E01300179
S315080049E032013401360139013B013D013F014101E4
S315080049F04301450147014A014C014E01500152014C
S31508004A005401560158015A015C015E0160016201B8
S31508004A106401660168016A016C016E017001720128
S31508004A207401760179017B017D019101910392035D
S31508004A3093039403950396039703980399039A039C
S31508004A409B039C039D039E039F03A003A103A3034B
S31508004A50A403A503A603A703A803A903AA0310048E
S31508004A601104120413041404150416041704180474
S31508004A7019041A041B041C041D041E041F04200424
S31508004A8021042204230424042504260427042804D4
S31508004A9029042A042B042C042D042E042F040104B3
S31508004AA002040304040405040604070408040904AC
S31508004AB00A040B040C040E040F0460216121622110
S31508004AC063216421652166216721682169216A219C
S31508004AD06B216C216D216E216F2121FF22FF23FF9F
S31508004AE024FF25FF26FF27FF28FF29FF2AFF2BFF84
S31508004AF02CFF2DFF2EFF2FFF30FF31FF32FF33FF34
S31508004B0034FF35FF36FF37FF38FF39FF3AFF00001D
S31508004B104F70656E424C54002E2E2F2E2E2F2E2EA1
S31508004B202F536F757263652F66696C652E63000077
S31508004B304669726D77617265207570646174652067
S31508004B4072657175657374206465746563746564EC
S31508004B500A0D00004F70656E696E67206669726D92
S31508004B60776172652066696C6520666F722072656A
S31508004B706164696E672E2E2E000000004552524F62
S31508004B80520A0D004F4B0A0D000000005374617263
S31508004B9074696E67207468652070726F6772616DDC
S31508004BA06D696E672073657175656E63650A0D00BC
S31508004BB050617273696E67206669726D7761726596
S31508004BC02066696C6520746F206F627461696E2057
S31508004BD065726173652073697A652E2E2E00000052
S31508004BE045726173696E672000000000206279745F
S31508004BF065732066726F6D206D656D6F72792061C1
S31508004C00742030780000000052656164696E672080
S31508004C106C696E652066726F6D2066696C652E2EEE
S31508004C202E4552524F520A0D00000000496E766119
S31508004C306C696420636865636B73756D20666F7550
S31508004C406E642E2E2E4552524F520A0D0000000059
S31508004C5050726F6772616D6D696E672000000000A3
S31508004C6020627974657320746F206D656D6F727933
S31508004C70206174203078000057726974696E672065
S31508004C8070726F6772616D20636865636B73756DAB
S31508004C902E2E2E00436C6F73696E67206669726DDF
S31508004CA0776172652066696C650A0D004669726DE2
S31508004CB077617265207570646174652073756363C6
S31508004CC065737366756C6C7920636F6D706C65744B
S31508004CD065640A0D000000002E2E2F2E2E2F2E2E74
S31508004CE02F536F757263652F41524D434D335F5392
S31508004CF0544D33322F756172742E630000600008BC
S31508004D0000200000030000000080000800200000CA
S31508004D100400000000A000080020000005000000B4
S31508004D2000C00008002000000600000000E000089F
S31508004D300020000007000000000001080020000015
S31508004D4008000000002001080020000009000000FB
S31508004D5000400108002000000A0000000060010869
S31508004D60002000000B000000008001080020000061
S31508004D700C00000000A00108002000000D00000043
S31508004D8000C00108002000000E00000000E0010835
S31508004D90002000000F0000002E2E2F2E2E2F2E2E64
S31508004DA02F536F757263652F41524D434D335F53D1
S31508004DB0544D33322F4743432F766563746F7273AE
S31508004DC02E630000002020202020202020202828D4
S31508004DD028282820202020202020202020202020AD
S31508004DE020202020208810101010101010101010ED
S31508004DF0101010101004040404040404040404101D
S31508004E0010101010101041414141414101010101AA
S31508004E100101010101010101010101010101010174
S31508004E201010101010104242424242420202020280
S31508004E300202020202020202020202020202020244
S31508004E4010101010200000000000000000000000F4
S31508004E500000000000000000000000000000000044
S31508004E600000000000000000000000000000000034
S31508004E700000000000000000000000000000000024
S31508004E800000000000000000000000000000000014
S31508004E900000000000000000000000000000000004
S31508004EA000000000000000000000000000000000F4
S31508004EB000000000000000000000000000000000E4
S30D08004EC00000000000000000DC
S30D08004EC801000000C44D0008BA
S70508000000F2
